:020000000328D3
:1000060030238312BD013D08BE00C2235008B7004D
:100016005008C800B023BD0A3708003AFF30031D58
:100026000030D1007F303D02FF30031C0030D0008D
:100036005108D004031D20280628BE01C2235008FB
:10004600BA008312051A39282D179F149F182928DC
:100056001E08BA00051E2D284430C800B0233E30C5
:10006600C800B023BE013A08BF004D233A08C700B6
:10007600AB213A08D000D1016430D400D501C322A7
:100086008130D4000030D50013235008A9002B304E
:10009600BE00EE225008B7002B08003A031DA12827
:1000A6003708BE0098235008B70050080D3A031DC4
:1000B6005E283B30B7002030BE008023003051065A
:1000C600031D672800305006031D87283708413A6C
:1000D600FF30031D0030D10037083B3AFF30031DC7
:1000E6000030D0005108D00403198628203084003F
:1000F600D32337088000840A800137083B3A031D62
:100106008628AD13A001A1282030BE008023003030
:100116005102031D902808305002031C9428A001A8
:10012600A12820308400D32337088000840A800168
:1001360037083B3A031DA128DB20A0012D1AA7286A
:1001460083129F142D16C02883129F18C0282D12C3
:10015600051EB0281E08AC00C028DF23051AC028DB
:100166009F149F18B4281E08AA00051EB8289622B8
:10017600DF232C08C700AB21AD17AD1FD7282C08ED
:100186003B020318C92805108514D62834082C020A
:100196000318D02805148510D6282C08C700AB21D3
:1001A60005108510AD13D928051085104A28DA28C0
:1001B60020308312C3004130BE004930BF003130C9
:1001C600C0003B30C100C2013E30C4000430C5004F
:1001D600C601162200305106031DF32800305006D2
:1001E600031DFE282C08C700AB212D1FFD282A0859
:1001F600C700AB21AA292030C3004130BE005030D1
:10020600BF003130C000C1013E30C4000330C5001C
:10021600C601162200305106031D13290030500670
:10022600031DAA290530AB000130BD00B201B301A0
:1002360003302B02031C55292B08203E8400303046
:100246000002FF30031C0030D1002B08203E840042
:100256000008393CFF30031C0030D0005108D0059F
:1002660003194B292B08203E840030300002D000B1
:100276000030031C013ED101D1023D08D400D50156
:10028600C3225008B20751080318013EB3074C2990
:10029600AA293D08D0000A30D40067235008BD00C3
:1002A600AB031B292D1B9C293308003C031D5D292C
:1002B6003208B43C03186429B430B202031CB303F9
:1002C6006829B430B2070318B30A00303302031D9D
:1002D6006E29B4303202031886293930D000003036
:1002E600D1003208D4003308D500C3226430D400CC
:1002F600D501132304305007B00051080318013EFE
:10030600003EB1009B290E30D0000030D1003208EB
:10031600D4003308D500C3226430D400D50113239A
:100326004D305007B00051080318013E003EB100A1
:10033600A0293208B0003308B1003008AA0096227E
:100346002D1FA8292C08C700AB21AD17AA29080024
:1003560083122D1BF929053047020318B529B2016E
:10036600B301E7292C08B000B10129084702031898
:10037600D2293008D0003108D1001230D400003024
:10038600D500C3220A30D400D5011323073050020A
:10039600B2000030031C013E5102B300E7293008C9
:1003A600D0003108D1004830D4000030D500C32237
:1003B6000A30D400D50113232C305002B20002308B
:1003C600031C013E5102B30000303302031DED2928
:1003D600B43032020318F429B430B2070318B30A52
:1003E600F829B430B202031CB303FC294708B20053
:1003F600B3013208C8003308C9002030CA005622AB
:100406000230AB0005302B020318112A2B08203EC0
:1004160084000008C800B023AB0A052A3B30C80098
:06042600B023A001080054
:10042C0083124308D8004408D90000304606031D47
:10043C00212A0030450603194F2A58088400000869
:10044C00D3005308D600590884000008D200520883
:10045C00D7005308003AFF30031D0030D100530879
:10046C005206FF3003190030D0005108D004031994
:10047C00482A57085602D4000030031C013ED5010F
:10048C00D502512A0130C502031CC603D80AD90A69
:10049C001B2AD401D5015408D0005508D1000800FE
:1004AC0083124A08840030308000840A3030800087
:1004BC00840A30308000840A30308000840A303066
:1004CC008000840A8001840A04304A07CB00003083
:1004DC004906031D732A003048060319952A0A3071
:1004EC00D400D5014808D0004908D100132358087E
:1004FC00D0005908D1003030D0074B088400500888
:10050C0080000A30D400D5014808D0004908D10039
:10051C0013235008C8005108C900CB036D2A0800EA
:10052C0083122A08023C031CA12A0230AA00B4013F
:10053C000430BB00B72A02303A02D10051082A021B
:10054C00031CB12A02303A02AA0004303A02B40069
:10055C003A08BB00B72A02302A02B40002302A073C
:10056C00BB002D1FC22A3408C700AB212A08C700C4
:0A057C00AB213B08C700AB210800CB
:1005860083120313DB01DA01D9018030D800D10CC4
:10059600D00C031CD72A5408D90755080318550F41
:1005A600DA070318DB0A0310D01FDF2A5408DA071C
:1005B60055080318550FDB07DB0CDA0CD90CD80CE1
:1005C600031CCA2A5B08D3005A08D2005908D10076
:0605D6005808D0000800E7
:1005DC0008308312B600B801851DFA2A3E08840043
:1005EC00FF308000BF01102BD923851D032B3E0843
:1005FC008400FF308000BF01102BCD23851D03101C
:10060C0085190314B80CB60B032B3808BF003E0831
:0A061C00840080013F08D0000800B0
:1006260083120313D801D9011030DC00510DD80D07
:10063600D90D5408D8025508031C550FD9020318C2
:100646002B2B5408D80755080318550FD907031044
:0A065600D00DD10DDC0B192B0800AC
:10066000831285018B010730990009309F008316A2
:10067000FF2390001C3085009F0104309F008C01F7
:100680009601950199010F308100831285019E0129
:0A069000AD01AC01AA0185160800B7
:10069A0083169C1C522B00004D2B3E089B003F08E2
:1006AA009A009C131C150B08D0008B1355309D0023
:1006BA00AA309D009C14D01B642B8B13652B8B17BF
:0406CA001C110800F7
:1006CE00831203135008D100D0010830DC0051080A
:1006DE00D40C0318762BDC0B6F2BD10100340310D6
:1006EE007B2BD40C0318D107D10CD00CDC0B782B40
:0206FE000800F2
:1007000083123E08D400540884000008003A0319FC
:100710008B2BD40A832B3E085402D200D301031C36
:10072000D3030030D3005208D0005308D100080092
:1007300083123E087A3CFF30031C0030D100613048
:100740003E02FF30031C0030D0005108D0050319D1
:10075000AB2BDF30BE053E08D2005208D0000800A7
:1007600008308312B6004808B5008512CD23B50CB9
:10077000031C851203188516CD23B60BB72B8516DF
:04078000CD2308007D
:1007840083123E0883169B009C131C141A08D10084
:060794005108D00008002E
:0C079A003230B9000000B90BCF2B080072
:0C07A60000080319D82B840AD32B08008C
:0C07B2000C30B9000000B90BDB2B080074
:0C07BE006430BC00CD23BC0BE12B080014
:02400E008431FB
:020000040000FA
:10420000FF000D000D0048005A0052006F007400BE
:104210006F0072002000560031002E003000200098
:104220004200750069006C00640028003000320014
:10423000360029002000620079002000500065004F
:10424000640072006F0020004C00550037004800E9
:104250005A00200032003000310032000D003B00D7
:104260000000FF00FF00FF00FF00FF00FF00FF0055
:10427000FF00FF00FF00FF00FF00FF00FF00FF0046
:10428000FF00FF00FF00FF00FF00FF00FF00FF0036
:10429000FF00FF00FF00FF00FF00FF00FF00FF0026
:1042A000FF00FF00FF00FF00FF00FF00FF00FF0016
:1042B000FF00FF00FF00FF00FF00FF00FF00FF0006
:1042C000FF00FF00FF00FF00FF00FF00FF00FF00F6
:1042D000FF00FF00FF00FF00FF00FF00FF00FF00E6
:1042E000FF00FF00FF00FF00FF00FF00FF00FF00D6
:1042F000FF00FF00FF00FF00FF00FF00FF00FF00C6
:00000001FF
